:100000000B28061E072882070734803482348207B3
:1000100007347F345634831613308500F030860061
:100020002730810083128501860183214630AA2171
:100030003630AA214230AA215130AA215530AA21B6
:100040002D30AA214630AA213530AA21C9215230AB
:10005000AA214430AA214830AA212030AA215630B2
:10006000AA213330AA212E30AA213030AA212830EB
:100070003421C1210430900086019D019E01861427
:10008000000086108101061586153921861106119A
:1000900001089C0083167030860083121C089300B0
:1000A0001308010603195D28000000000310FF304B
:1000B00093001D0813029D00622886170000861316
:1000C0009D0A50288316F03086008312861F7B28F5
:1000D000861B7628000000000310FF3093001E08E6
:1000E00013029E009E0A03189D0A80289E0A061588
:1000F0000000061168289E0A0615000006116628F1
:10010000061FD128861EB0288528930102300120C1
:1001100003149E0203189728031401309D0203184C
:100120009728031401309C020318972813140130F8
:10013000012003149D020318A328031401309C021C
:100140000318A32813140301012003149C020318AD
:10015000AA28AC28131CD1289E099D099C09D128E6
:1001600093010230012003109E07031CC2280310D4
:1001700001309D07031CC228031001309C07031C9B
:10018000C22813140130012003109D07031CCE2840
:10019000031001309C07031CCE2813140301012017
:1001A0009C071E0899001D089A001C089B00900BD4
:1001B0003C28023090005A21C5213030930022089B
:1001C0000F39031DE6282030AA21E8281307AA21A9
:1001D000210E0F391307AA212E30AA2121080F3929
:1001E0001307AA21200E0F391307AA2120080F395F
:1001F0001307AA212E30AA211F0E0F391307AA2197
:10020000C9212030AA214D30AA214830AA215A30D4
:10021000AA212030AA21061F282905181F29851C7C
:1002200018295530AA215330AA214230AA212E295B
:100230002030AA214330AA215730AA212E2985181F
:1002400028294C30AA215330AA214230AA212E2934
:100250002030AA212030AA212030AA211F080F39DE
:1002600013079100C5213C2897003921970B3529A8
:1002700000342D3094000C3095003C309600960BE5
:100280003F29950B3D29940B3B2996309400940B04
:10029000472900000000003442309400940B4E299E
:1002A00000340A30940042309500950B5529940B88
:1002B000532900340310183092009F01A001A101BE
:1002C000A2019E0D9D0D9C0D9F0DA00DA10DA20DD7
:1002D000920B6B2900342230840078212130840075
:1002E00078212030840078211F3084007821612912
:1002F000033000079300931980003030000793000B
:10030000931B8000003439218511051103308600CC
:100310000515000005113921033086000515000080
:1003200005114C21033086000515000005114C21F4
:10033000023086000515000005114C210C30A82163
:100340004C210630A8214C210130A8215121003434
:100350008511AB2985159800180E0F3986000515F3
:100360000000051142309400940BB42918080F398D
:10037000860005150000051142309400940BBE293B
:1003800000340130A821512100340230A82151212C
:0A0390000034C030A8214C210034D5
:02400E00FA3F77
:00000001FF
